:020000040000FA
:10000000B6017D29A4003A0884003808E020841352
:1000100000052C1C3806031920282408031D182865
:100020002A08FF3E031C21283230F4202A08212808
:10003000240AFF3003192028240B20282B0821280C
:10004000AD09AD0C7829B616B61EB61236192D2894
:10005000FE39B700361503107829361A3528A60060
:1000600036164C2003183A282608532003183A283D
:10007000B61E782945206A2036113612B6113A0884
:1000800084003808841780044B283A088400380913
:1000900080058417800508003F206A2045206620DF
:1000A0003708B6190138A2000830A300A20D0318C2
:1000B0003F20031C45206A206620A30B56283F20C2
:1000C0006A203A08840038080005FF3E3B08840097
:1000D000390948283B088400390880048417390905
:1000E00080054B28A501A400B7172730A3001030C6
:1000F00085200330A300E8308520A30164308520EB
:10010000A3010A30852024089028A2002508A10018
:100110002408A00046212008031DB713B71B0800C0
:10012000303EA7000611861186118316061186112E
:1001300086110F30860583122708B618BD283A307D
:10014000A100983002213330A600D1201330A10045
:1001500088300221D12064300121D1206430012176
:100160002230A600D1202830BC200C30BC20063024
:10017000BC20B6142708BD283614A600361CCB2890
:100180008611033C031CD028D0200730A100D030BA
:100190000221031408003614FE3C03197829861541
:1001A000361C361006150F3086052608F0398604F1
:1001B0000611A60E3618D12832300121031408008A
:1001C00084178004782983169B001C141A08782948
:1001D00083169A001C1555309D00AA309D009C1472
:1001E0009C18F0281C117829A301A200FF30A20757
:1001F000031CA307031C78290330A100DF30022170
:10020000F628A101E83EA000A109FC30031C0B293F
:10021000A00703180829A0076400A10F08292018C7
:100220001129A01C15290000152908000310A00D94
:10023000A10DFF3E03181629200878290310A10CF0
:10024000A00CFF3E03181E2920087829A101A30154
:10025000A20002302F29A101A301A2000530A800AD
:1002600023082102031D3629220820020430031826
:100270000130031902302805031DFF3078290038AA
:10028000031DFF300405031DFF307829A501A401DB
:100290001030A600210DA40DA50D2208A4022308EC
:1002A000031C230FA50203185C292208A4072308B6
:1002B0000318230FA5070310A00DA10DA60B4A29B3
:1002C000200878291030A800A101A001A70CA60CD5
:1002D000031C70292208A00723080318230FA10775
:1002E000A10CA00CA50CA40CA80B66292408782945
:1002F0008313031383126400080083160515851504
:1003000005160614831207309F0064006430F42041
:10031000D401D7016400051D3F2CFE30912001302F
:10032000912041309120563091202D3091204D3038
:100330009120613091207430912072309120693089
:10034000912078309120203091205630912030300B
:1003500091202E3091203130912065309120FE3057
:100360009120C0309120543091206F3091206D3019
:100370009120743091206F3091206D309120203089
:100380009120443091204C309120313091204D30DB
:100390009120463091204B3091200530A300DC3075
:1003A000F520882C0530BA000430B800AC01FF30CD
:1003B000AA00AB010130AD004E080220CE000318A8
:1003C0000F2A0530BA000830B800AC01FF30AA008F
:1003D000AB010130AD004F080220CF000318192AED
:1003E0000530BA001030B800AC01FF30AA00AB01F4
:1003F0000130AD0050080220D00003181C2A06303E
:10040000BA000130B800AC01FF30AA00AB010130E6
:10041000AD0051080220D10003181F2AD229D201B1
:1004200055106400061C7A2E64008519182A55148C
:10043000242A0130D200242A0230D200242A033098
:10044000D2006400051D7A2E0030D5180130A000BE
:1004500001302621B2005208A00000302B21B40048
:100460003208840034083F21B400B5006400340829
:1004700035040319412A5208403E84004008800098
:100480005F2A5208403E84000008B2000130320763
:10049000B200B301B30D5208403E84003208800020
:1004A0005208403E84000008B20064000D30320261
:1004B000031C5F2A5208403E84000130800052082D
:1004C0003C3E84000008B200FF303207B200FF302B
:1004D0000318013EB3003208A0003308A100043025
:1004E000A200A3014621CD004D08A600A7010230BD
:1004F000A200A3016221B2002508B30090303207A8
:10050000D6004D08473E84000008B2000130A0002C
:10051000A10152081921B4002108B5003208B40421
:100520004D08473E8400340880004D08473E840053
:100530000008B2000130A000A10152081921B40046
:100540002108B5003208B4064D08473E840034083F
:1005500080000530BA000130B8000530BB00023021
:10056000B90056082520023025204D08473E84005A
:100570000008B200320823205208403E84000008E0
:10058000B200FF303207B200FF300318013EB30063
:100590003208A0003308A1000430A200A3014621C4
:1005A000CD004D08A600A7010230A200A3016221E0
:1005B000B2002508B30090303207D6005208403E02
:1005C00084000008B2004D08A600A7010430A20074
:1005D000A3016221B4002508B50034083202B4003A
:1005E00035090318013EB5003403D3004D084A3ED7
:1005F00084000008B2005208A600A7010230A20041
:10060000A3016221B4002508B5000330A000A101B8
:1006100034081921B4002108B5003208B4044D088B
:100620004A3E8400340880004D084A3E8400000899
:10063000B2005208A600A7010230A200A301622165
:10064000B4002508B5000330A000A1013408192129
:10065000B4002108B5003208B4064D084A3E8400B3
:10066000340880004D084A3E84000008B200520859
:10067000A600A7010230A200A3016221B400250850
:10068000B5005308A000A10134081921B4002108C5
:10069000B5003208B4070318B50A4D084A3E840075
:1006A000340880000530BA000130B8000530BB00C6
:1006B0000230B90056082520003025204D084A3E5A
:1006C00084000008B200320823206400551C952BDA
:1006D0004D08443E84000008B20004305307B400C3
:1006E000B501B50D0130A000A10134081921B400F5
:1006F0002108B5003208B4064D08443E8400340891
:1007000080000530BA000130B8000530BB0002306F
:10071000B90056082520013025204D08443E8400AC
:100720000008B2003208252055104D08473E8400CD
:100730000008B2000130A000A10152081921B40044
:100740002108B5003208B4044D08473E840034083F
:1007500080000530BA000130B8000530BB0002301F
:10076000B90056082520023025204D08473E840058
:100770000008B200320823205208403E84000008DE
:10078000B20052083C3E840032088000D70100309D
:100790005707B200B301B30D320883169B008312D2
:1007A0004A08E82001305707B200B301B30D320800
:1007B00083169B0083124B08E82002305707B200D3
:1007C000B301B30D320883169B0083124C08E82056
:1007D00003305707B200B301B30D320883169B00F4
:1007E00083124408E82004305707B200B301B30D68
:1007F000320883169B0083124508E820053057070E
:10080000B200B301B30D320883169B008312460871
:10081000E82006305707B200B301B30D3208831643
:100820009B0083124708E82007305707B200B30146
:10083000B30D320883169B0083124808E820083065
:100840005707B200B301B30D320883169B00831221
:100850004908E82009305707B200B301B30D320848
:1008600083169B0083120030D5180130E820640005
:100870005408003C03193E2CD401DC2C0E2E093008
:10088000E32001390319D510031DD5148310D51C9D
:1008900083148318D514831CD510FE3091200130A9
:1008A0009120563091206F30912072309120773016
:1008B000912061309120683091206C309120FE3081
:1008C0009120C03091206400D518722C4E309120B8
:1008D00069309120633091206830912074309120EC
:1008E00020309120413091204B3091205430912084
:1008F00049309120563091200530A300DC30F5209E
:10090000831609309B0083120030D5180130E8208F
:1009100000305707B200B301B30D3208E320CA001C
:1009200001305707B200B301B30D3208E320CB000A
:1009300002305707B200B301B30D3208E320CC00F8
:1009400003305707B200B301B30D3208E320C400EF
:1009500004305707B200B301B30D3208E320C500DD
:1009600005305707B200B301B30D3208E320C600CB
:1009700006305707B200B301B30D3208E320C700B9
:1009800007305707B200B301B30D3208E320C800A7
:1009900008305707B200B301B30D3208E320C90095
:1009A00009305707B200B301B30D3208E320013913
:1009B0000319D510031DD514D2016400033052026F
:1009C00003182A2D0230A600A7015208A200A30195
:1009D0006221B2002508B30090303207D6000530FE
:1009E000BA000130B8000530BB000230B90056082B
:1009F00025200030252052084A3E84000008B2001D
:100A0000320823200530BA000130B8000530BB00A1
:100A10000230B90056082520013025205208443EF6
:100A200084000008B200320823200530BA000130EB
:100A3000B8000530BB000230B9005608252002304E
:100A400025205208473E84000008B20032082320C7
:100A5000D20FDD2CD2016400033052020318092E9C
:100A60005208473E84000008B20001303205B2004F
:100A7000B3013208A0003308A100A30101302D21E9
:100A8000031D5F2D52084A3E84000008B200033067
:100A90003205B200B3015208A600A7010430A2003B
:100AA000A3016221B4002508B5003208B407330859
:100AB0000318013EB507340AC0004008BC005208C4
:100AC000473E84000008B20002303205B200B30194
:100AD0003208A0003308A100A30102302D21031D1C
:100AE000972D52084A3E84000008B2000C303205AF
:100AF000B200B3013208A0003308A1000230212166
:100B0000B2002108B3005208A600A7010430A200D9
:100B1000A3016221B4002508B5003208B4073308E8
:100B20000318013EB507340AC1004108BD00520850
:100B3000473E84000008B20004303205B200B30121
:100B40003208A0003308A100A30104302D21031DA9
:100B5000CF2D52084A3E84000008B20030303205E2
:100B6000B200B3013208A0003308A10004302121F3
:100B7000B2002108B3005208A600A7010430A20069
:100B8000A3016221B4002508B5003208B407330878
:100B90000318013EB507340AC2004208BE005208DD
:100BA000473E84000008B20008303205B200B301AD
:100BB0003208A0003308A100A30108302D21031D35
:100BC000072E52084A3E84000008B200C0303205A9
:100BD000B200B3013208A0003308A1000630212181
:100BE000B2002108B3005208A600A7010430A200F9
:100BF000A3016221B4002508B5003208B407330808
:100C00000318013EB507340AC3004308BF00D20FE2
:100C10002B2D64005408003C031D8C2FFE309120C6
:100C2000013091204F309120753091207430912007
:100C3000313091202030912020309120203091209F
:100C4000323091202030912020309120203091208E
:100C5000333091202030912020309120203091207D
:100C600034309120FE309120C030912049309120C5
:100C70006E30912020309120D20164000430520265
:100C80000318792EFE3091205208A600A7010430E7
:100C9000A200A3016221B2002508B300C330B2074D
:100CA0000318B30A320891205208403E840000081D
:100CB000B20064000A303202031C702EFE30912014
:100CC0005208A600A7010430A200A3016221B200CD
:100CD0002508B300C230B2070318B30A32089120C6
:100CE0005208403E84000008B20032087220D20F41
:100CF0003D2ED229FE309120013091205330912099
:100D000065309120743091207530912070309120A1
:100D1000FE309120C03091205330912061309120DD
:100D20007630912065309120203091202030912024
:100D300020309120203091202030912020309120AF
:100D40002030912020309120523091206530912028
:100D500061309120643091200530BA000430B80031
:100D6000AC01FF30AA00AB010130AD004E080220FB
:100D7000CE000318E92E0530BA000830B800AC01E7
:100D8000FF30AA00AB010130AD004F080220CF00B8
:100D90000318E92E0530BA001030B800AC01FF305E
:100DA000AA00AB010130AD0050080220D0000318AA
:100DB0006F2F0630BA000130B800AC01FF30AA0036
:100DC000AB010130AD0051080220D10003186F2F94
:100DD000AC2EFE30912001309120533091206130B3
:100DE00091207630912065309120203091204D3037
:100DF00091206F3091206430912065309120FE3039
:100E00009120C03091200130D400FE309120C030BC
:100E100091205408722020309120203091202030E1
:100E20009120203091202030912045309120783041
:100E300091206930912074309120203091205330DE
:100E400091206130912076309120653091200530DD
:100E5000BA000430B800AC01FF30AA00AB01013089
:100E6000AD004E080220CE000318552F0530BA0001
:100E70001030B800AC01FF30AA00AB010130AD006A
:100E800051080220D10003185E2F0630BA0001304D
:100E9000B800AC01FF30AA00AB010130AD00510831
:100EA0000220D1000318602F272FD40A64000A30D3
:100EB0005402031C5D2F0130D400052FD4010E2EE7
:100EC0005408A600A7010930A200A3016221B200C4
:100ED0002508B30003303207D700D401C72BFE30FA
:100EE0009120013091205230912065309120613065
:100EF000912064309120203091204D3091206F302E
:100F000091206430912065309120FE309120C030D6
:100F100091200130D400D701FE309120C0309120C3
:100F200054087220203091202030912020309120D0
:100F30002030912020309120453091207830912030
:100F400069309120743091202030912054309120CC
:100F5000613091206B309120653091200530BA00CE
:100F60000430B800AC01FF30AA00AB010130AD0085
:100F70004E080220CE000318DF2F0530BA001030D3
:100F8000B800AC01FF30AA00AB010130AD00510840
:100F90000220D1000318DC2F0630BA000130B8005F
:100FA000AC01FF30AA00AB010130AD0051080220B6
:100FB000D1000318F52FAE2FD401D701882CD40A05
:100FC00064000A305402031CE72F0130D400540897
:100FD000A600A7010930A200A3016221B2002508E2
:0E0FE000B30003303207D700882CD701C72B8F
:02400E00183F59
:1042000000000000000000000000000001000200AB
:044210000C0000009E
:00000001FF
